:10000000020A9CD2D3FA20B25A0526201F3DDB44B7
:1000100001E400C2AA30075B01C700106247200755
:100020006301B9109919C0E0E59964607012C2AA21
:10003000C295758BAF758DFE432C24C298D0E032EB
:1000400030E604C2AC013DC223013BAE8CE4F58A2C
:10005000F58C01FAEB20E04C202441E5287002D217
:1000600027152801A4D29530B45220653B758DF434
:10007000D2AC32C295D294D262758B29758DFFC2F3
:100080008FD2AB3220600D30B351D2607531027522
:100090008DBF01C2D53104C2ABC260320528E5284C
:1000A0007002D227EAC2D332758DDB302F0A2023AB
:1000B00007759970C22FD22332306506C2ACC26573
:1000C000C2ABC28BD2AA32054B75360310600875DD
:1000D0008B00758DFF017F054901CF054AD536EFAD
:1000E0007522B332D292C290EDF2E3FE74CCF2AB41
:1000F0000C748CF2306403639005D21EEAC2D332D2
:10010000314AFA30D52530980BE599601EE59931D2
:100110004A1098F98A997540FA10980A3156DBF915
:10012000D540F6C2D522E599B440E222758C00C2D2
:100130008D208DEF3098FA3098FDC298E599FB201C
:10014000E602F599532020D2D5227B3CDBFE22C269
:10015000A6432F21C23E303E0D308D0AC28DDD06F2
:10016000B27DAD0FD23EC264D292C2907803E52F29
:10017000F222C264D292C2907801E2C52D22927B13
:10018000B3927CAB164002AB17020ECCF522750F72
:10019000077C023162300016D2A621AE3172C20B4A
:1001A000306B02D20BE5212100319C30170D30D588
:1001B0000AE5223100E53ED2E73100315610983091
:1001C00030170B3172652D30E2F1DCEF0100200AAF
:1001D00057315151F11098187488203705306C044C
:1001E00074A74190206A053000D161A9C23F61E443
:1001F000313A20E6C67F0324F6502724E5500474E4
:100200009B218C301704748B218C300A08241960D0
:1002100004749C218CC2A6C2AF7A0851E93027022F
:10022000F164900317EB2B733172206F14300808C0
:10023000206A0C203F0B810E51CF751100B1DBC23B
:100240003FD2AF51CF20374F306F06E52624EC4028
:100250000851D66002B27821BBC23F751112B1DBE2
:100260007A4610083A314F20372D51E23172206F13
:10027000F605120511B1DB7F06C28FE52624E340A7
:100280001A308FF751E2DFF1DAE77487F53E7489AF
:10029000F522314F020C897494418CD20861F751D8
:1002A000C4C28F20B515203712E526B41D00308F4B
:1002B000FD40066526600851E2DAE6748A419075D1
:1002C000122661FD532FDE7551FF316602095AB2C5
:1002D00078D550021551E55154F06003316622C2C1
:1002E000782210980122E599227941E4F709DAFB96
:1002F000223172652D20E21220E3097440100111B1
:10030000206A1022319CC20B6113306AEEE5214451
:100310003031027B0241CC0100616D21A961756120
:100320007E61806184618E21B1619881B3619C811D
:100330000C61BA61BC61D261D461D661E0810C818B
:100340003E813F8193A123A12421BBA142A144A1CD
:1003500056A155A15AA170A178A17AA17EA184A12C
:1003600082A18BA18D312CF525D201A16B740D31A9
:1003700000E54E21B9E4F522F53EC2D521BB79FF57
:1003800009E721B9792AE7310019DFFA21BB792A77
:10039000312CF719DFFA21BB794B6186120EC5E4C7
:1003A000F53BC2A43098FD21BBE52B0430E012756B
:1003B00024057539F6753A0081BAD203C2D5D20048
:1003C000E4752415753AE17539F3B416EB10031092
:1003D00061D4D266D202432130F12120173F81132C
:1003E000D23FC2D5200AC061D6D23D741081BAC2B4
:1003F00024120A06201726120A6F201720B1DB5399
:10040000210FD20A51C48B2651E28133C23F300002
:1004100002D202D224314F120A0630170241927AD8
:1004200003792851EBC227206ABF203FBC20020776
:10043000200089D2A621A97A0B51E9020CE0D392BF
:1004400024D22081B353130C20000720B404749EDF
:10045000218C53210FD20D1208EDB1D5B190201788
:100460003030B52B3000033020273098EFE599303D
:10047000E60C20ACE7C29820E5E2C223815CFB24B5
:10048000E624F2400CC298781ED8FE8B994122D205
:1004900026A144532480783A792A7A02312CF40434
:1004A000F620200B27600843240530E702D22418E9
:1004B00019DAE9312C30D54DD201C2097002D209C6
:1004C000FEC313FF317EC22CEEC52BFEC313C39FA8
:1004D0005004D22CF404FC60047D13D221EE652B71
:1004E00014602920E00EE53B20581C302C02F40457
:1004F0002DFDD221103D0C202007D220205802D201
:1005000024814561EF21BB202CE681EEFDE53B60B7
:10051000E30C20580930E7D9F404D22C81F120E70C
:10052000CDA11AD39224B2241208EDB1D57B1EB10D
:1005300090201710301BF8308DF5C28DDBF1D20101
:10054000A144D2041209672017031004D912099795
:100550003017B24192D3317EA16B300B0575229DCD
:10056000A16BD205301B04C2A4C274201CE2815CC2
:10057000D2A4D274C205A16BD207D294A16BD2953A
:10058000A16BD23C53A881C207A16B1D1D0DA16BAD
:10059000101E02E164E50E30E702747E24E0FA20CA
:1005A0001951201848E50E20E00D24E850091025C7
:1005B00004D225A1B9C1EDC225758D29DF2E7F0298
:1005C00078117912E51D2024040819E51927401C2B
:1005D00007E6600716E52E4513F5A0D2AFD264D228
:1005E000905390F3E511F2D293E512F2220523E441
:1005F000F552FED21DEAC530F4042AC333255279E0
:1006000015D188CA301F087906D1882AFAC1262E4A
:10061000C330E704046002D313FEDF0A7F036006E1
:1006200020E7020A0A1AEA60C378028537F0C21A84
:1006300030E704D21AF404F614600312095078115A
:100640007912202407201A070819C14F201AF9EA45
:10065000264031F6301A04253F4029E79A600250BF
:10066000052614F67401F7301F18E52A54F87012A5
:10067000E512202404793CD188B41300500274148C
:10068000F512A1DB75228722F875520020E708C316
:1006900099400CF552E922294005F552E49922E8E7
:1006A00022101E05308FE0E11D758D29DB02154DEE
:1006B000302108EB540370031208B1108DC9E50E08
:1006C0007996D18875520024C820E70EFA2530505B
:1006D0000824D85004F4042AFAEAF404FA3019027F
:1006E000A1F3301802A1EDE50E24C2409A05238A39
:1006F00030851A11851E12758D9EC28F752E93A19D
:10070000D5208D16E526CF6F6003758CD220275437
:10071000308F09C28FDA0575228CD21C2275228691
:10072000227C08C2035324E01208ED750F50D23E1C
:10073000B1D5B19020172730B51831563098F3E570
:1007400099C298B402ECF599D2D5314A8521992005
:10075000B5E02054DD752A008528548529551209F5
:1007600067020997102761201B2F201909208FADE0
:1007700030214C0208A92021FA200205431320D27F
:10078000A530030D30A40DC2A4758D9E20B431C2D6
:100790008F102F30308F28D21B30224D20204D302B
:1007A0000504C2A4C2747A402023145324F03001FB
:1007B0000E200704C28BD2AA30D504D2238A9922F4
:1007C00075229F227A70E1B87929200002B2A62012
:1007D000244317304F501528771109173057410718
:1007E000300C02DC03752298222020B320650620FD
:1007F0002303102FCF101D612006102003063007A1
:10080000543095104320C0C28BD2AAE54B24065029
:10081000037522B22207B7120D7700090720553160
:10082000153F153F313130221130200EE52A253A8F
:100830007008E52925397002C220200C137A0BE5D7
:100840002A6004B41F0A0AEAB52905300102D22F32
:10085000221775229720285122EE30E702F404F582
:100860001024E4501C20630BD26375531E300C031C
:1008700075530220B404C295D2A4D55303752299AE
:1008800022C263300502C2A4303CCA781079427A91
:1008900003E6C397E64001F70927F7095001070867
:1008A000E6DAF5D54146C23C22308D40758C64C2F3
:1008B0008D202929E51423302C020303F514540C50
:1008C000F513452EF5A0202809DD21DC1D7D06D27B
:1008D00029220515202CF81515151501CF1028050E
:1008E000200202DD07C221C229227D1322752E9229
:1008F0007918E52AC403202405152EF4791C54F830
:10090000F8900F00314320240279183143851811E3
:10091000851C12051E051E85193F202403851D3FD9
:100920007404F50BF50CFFE4F58CF58DF523538875
:100930005F75371AE52A202402641F24F6400375E8
:100940003713227A04E893F70809DAF92275F00FD1
:10095000E6A4C4F6E5F0C4D6F6227B28758C64C202
:100960008D308DFDDBF62253A8815390CF5324F2B6
:1009700053201F11ED851B11851F12532CD07A06B1
:10098000752E91202402052E1205D512070120B5DF
:1009900002D226301CF522D21C781275F010E52AFE
:1009A00023B41900400303240D2425103812D23833
:1009B000302404240405F0F63150E52A641F21A0F8
:1009C00020240104F5111206FC7AFA30210411A941
:1009D00021CB758D64C28F752600308FFDE52660B2
:1009E00008DAEF85223E752288302703120764C299
:1009F000A610260620170E0202F1200C087522957B
:100A0000205402052222754D0A75290911ED781A24
:100A100075F00B3150781E75F00B31507537167B21
:100A200000C225D21F1205D5E58D30E5FB1206A1C7
:100A3000E54D30B51720170F30E7F2102509752264
:100A4000812024037522823197C21F222025DE20B7
:100A50000D0B20240470D6414754FC70D02054E77D
:100A600053210BD20CE4FBF54DF52AD225412D750F
:100A70001214751116D1DE76067526007A7871E1AA
:100A80007B05315CD1DE24F6400A2037070511DAF8
:100A9000ED30B504E52170AC7512192275A8017509
:100AA000891075885575B80175989A75815A759031
:100AB000CE75A0B37900748CF379087A521202EBE8
:100AC0001205DD752FF712016608745BF2087401D8
:100AD000F2E4F8E8F5F0C291F2E2D291B5F01CD858
:100AE000F2120172900000E4936AFAA3AC83BC0F87
:100AF000F66012748E41FD74A841FD7490F5228158
:100B0000AA749141FD750904750D4C751433D1C556
:100B1000120172452D20E6277912307C0719B29414
:100B2000D22811A90B315CA7021205D5DAEA632F8E
:100B3000FF7B32D1CC307CE0632E53B22C6118089D
:100B4000E2F54E30E7B120E50205207A14758B629C
:100B5000758DFDC28FD2D31200E4308FFDD2D31237
:100B600000E4E50E24F824CE4097DAE17D027535E5
:100B700003752B10D1A9315A8B268B2A8B2279121F
:100B8000D1DE760575110C7C647F0177258C8DC2D2
:100B90008F71E130B516D1DE30E7028111B40C005F
:100BA0005060203907B403048B26D239E526203B58
:100BB0003324FE401B308FDB103806770CD23861AF
:100BC0008F7CD9DFC60D30B53D202B04D22B618B35
:100BD0008B2620B502DD2FD23B771287117F8261F1
:100BE0008D0205DBB4F0005021308FA77C64CE6EFF
:100BF000709B07E724B0500330B55BDF9075112878
:100C0000516F7483818574AA8185E6600474A9811B
:100C100085303BF2E526B4460040EB94645001E495
:100C200020E7071313F4541FF52A3197D1A974282C
:100C30002511FFD1DE76FFE51224E65002151205DC
:100C40001171E1758D64C28FD1DE30E72C308FF8E1
:100C5000DFE574848185E52624E640F6315A20B527
:100C6000F18B117726053571E1315C20B58FD1B953
:100C7000F511F525D23F0202BFD1B9752410319785
:100C800030172C748DF522D22B7F647812314D18D9
:100C9000314D71E17B06315CDFF18F27302B0BD5B5
:100CA000350BD2087483652260C402018E6171D253
:100CB000085106E5226003B481CBD1B9F525431371
:100CC000200203D681F6A1CAA119A189A1F1C128E8
:100CD000C13AC177C158C169C16EC170C17081F696
:100CE0002066F17534FE7C10D22CD1B9F50FF53D9C
:100CF000F53BD1C5A1D0D1B9F534D224C22C754071
:100D000064202D08202A09202E047C06A1D0C224AC
:100D1000D22C7C03754055C122202848203B26C296
:100D20002C302D02C27430B329203904D2397B080B
:100D3000308F31DB2A202D3E202C3B203B0FD23B35
:100D400085153BA152202CDE20B307A129D22C759A
:100D50004014C239D54006302D0C7522A5D2287515
:100D60008DECC28FA1FA202A0F050F303B037522AC
:100D7000A0D22A7534FEA1F8E50F70057522A1C135
:100D800018203BF875340EA1F8102D2EE53BC395C5
:100D90001513FDD22C24F0240B400874A2207C01F2
:100DA0000441FD302E24E51524392D202404F5338B
:100DB000A1B4F53CF4042DFDA1CAE515F53D047080
:100DC0000474A641FD7C0775341005340534D23A0D
:100DD000B2244324057539F9D33024047539FEC390
:100DE00012017EEC6004D2217D1311ED1205D5A114
:100DF000FA202806D228DD02C23A120590201718E0
:100E000030B5132022F4E529C2E314600B303AEA2E
:100E1000900CC4E53473D22612075E301702818924
:100E2000C23A05340534C11075340A74052024040F
:100E3000F516C136F517F50FA1CA308FBD12017234
:100E4000206DB57B01050FD1D3743BB50F0875221A
:100E500092207CC40522A15F7525607450120100A8
:100E6000315A749F20B43781E37D07753414A1F1A2
:100E700010662FD205A1D030240A850F16750F00F9
:100E8000D22A81F6850F17E4202E15F53CE51524AE
:100E900039F53B30E702F40424F0500674A441FD18
:100EA000F53BC202752B0B81BA10980122E599B46B
:100EB00002FAF599D2D50201A5E4F524F53AF52711
:100EC000F515F5222275161675171622D27912011C
:100ED00066C279120166B27A307AF8DBF622120124
:100EE000727840E52D5403C50FB50F02C1F70365B5
:100EF0000F1630E0020606E622FFFFFFFFFFFFD3DA
:100F0000304360BF865B4C1B30415FC1875A4F192D
:100F10002F3F5EC3885952182E3D5CC38858551721
:100F20002D3B5BC489575816323959C48F515B1613
:100F3000313758C4904F5E16303556C4914E611605
:100F4000343355C497476317323153C399466617F4
:100F5000312F52C29A446818372D50C1A33B6B19E8
:100F6000362B4EC0A43A6D1A34294DBFA6386F1CDB
:100F700033274BBDA736721D312549BBA935741FD8
:100F8000302348BAAA3476202F2146B8AC327822D2
:100F90002D1F44B6AD317A242C1D42B5AE307C26CF
:100FA0002B1B40B3AF2F7E282A193EB1B02E8029CB
:100FB00029173CAFB12E822B29153AADB22D842DC5
:100FC000281338ACB22D852E281136AAB32D8730C0
:100FD000270F34A9B32D8931270D31A8B32D8B32BA
:100FE000270B2FA7B32D8D3328092CA6B22E8E34B4
:100FF000280729A6B22F9034290527A7B1309234AB
:00000001FF
